:030000000200B843
:0200030001A753
:02000B00011ED4
:10001B000200B8758CFF758A37307802B2970535B8
:10002B000536C530146003C530327464C530C0E08A
:10003B00C082C083C0D0D2D3B296D27D30790CC2ED
:10004B0095C2797533FF75340A8002D295307A06E2
:10005B00C294C27A8002D294C5332078086008B467
:10006B00FF02800114B278C533C5311470067404D5
:10007B00C5318002C531C5321470167414C532C235
:10008B007DE53470057533008005153475330480B8
:10009B0002C532D0D0D083D082D0E032C0E0C08253
:1000AB00C083C0D0D0D0D083D082D0E03275811045
:1000BB00752F007530647531047532147533027504
:1000CB003400753500753600758CFF758A37758968
:1000DB00117588118502B8D2A9D2AFA27D92932057
:1000EB00791D207B0A20B017D27B7535008010302C
:1000FB00B004C27B8009E535C394284002D2792035
:10010B007A1D207C0A20B117D27C75360080103006
:10011B00B104C27C8009E536C394284002D27A022E
:02012B0000E6EC
:00000001FF
